:03800000028011EA
:20800B00438CDC05083275810890F00CE4F0438901D2AFD2A9D28C1283B202195405817931
:20802B00027A0089828A83E0548078FE12865AF6700302805EE612868C7BFF128683128704
:20804B005D45F0700302805B74FF75F0FF02806302802A740175F000158122128028790006
:20806B007A00740189828A83F0221280287BFF7CFF12875D45F0700302808E74FF75F0FFA8
:20808B000280C779007A00743889828A83F012802879007A00740C89828A83F01280667444
:2080AB000075F000C0E0C0F0740075F000C0E0C0F01280C815811581158115812212802849
:2080CB0078FB12865AE612868C90812A02869579007A0078F912865AE6248089828A83F0E6
:2080EB0002813E79007A0078F912865AE624C089828A83F002813E79007A0078F912865A75
:20810B00E6249489828A83F002813E79007A0078F912865AE624D489828A83F002813E16DA
:20812B0081030002810200EE800100DA80000000003E81220581740078FE12865AF678FEB3
:20814B0012865AE618181818860108860275F00012867C89828A83E012868C7B001286839A
:20816B0012876645F070030281AF800B78FE12865AE604F61480C712802879017A00C0017E
:20818B00C00278FC12865AE618181818860108860275F00012867C89828A83E0D083D08239
:2081AB00F002817778FA12865AE60886F015812212802879017A0078FB12865AE689828ABC
:2081CB0083F0227F0812866678F312865AE60886F07B007C0012873D45F070030281FD7450
:2081EB000075F00079F712865F12867C742DF702820D740075F00079F712865F12867C74A3
:20820B002BF778F312865AE60886F078FD12865AF608A6F078F312865AE60886F07B007CBD
:20822B000012873D45F0700302825B78FD12865AE60886F012873678F312865AF608A6F04B
:20824B0018E60886F012872318F608A6F012872C740175F00079F712865F12867C78F31298
:20826B00865AE60886F07BE87C031286C52430C5F03400C5F0F718E60886F07BE87C031217
:20828B0086BE78FD12865AF608A6F0740275F00079F712865F12867C78FD12865AE6088663
:2082AB00F07B647C001286C52430C5F03400C5F0F778F312865AE60886F07B647C0012866E
:2082CB00BE78FD12865AF608A6F0740375F00079F712865F12867C78FD12865AE60886F0B8
:2082EB007B0A7C001286C52430C5F03400C5F0F7740475F00079F712865F12867C78FD124D
:20830B00865AE60886F07B0A7C001286BE2430C5F03400C5F0F7740075F00079F712865F8E
:20832B0012867CE712868CC0E0C0F01281BB15811581740175F00079F712865F12867CE70D
:20834B0012868CC0E0C0F01281BB15811581740275F00079F712865F12867CE712868CC003
:20836B00E0C0F01281BB15811581740375F00079F712865F12867CE712868CC0E0C0F01224
:20838B0081BB15811581740475F00079F712865F12867CE712868CC0E0C0F01281BB1581D3
:2083AB0015817FF8028675746475F000C0E0C0F01284CF1581158112807574B875F087C0AB
:2083CB00E0C0F012813F15811581740075F000C0E0C0F0740175F000C0E0C0F01280C81542
:2083EB008115811581158174C875F087C0E0C0F012813F1581158174C875F000C0E0C0F0C8
:20840B001284CF15811581740075F000C0E0C0F0740175F000C0E0C0F01280C815811581E7
:20842B001581158174D875F087C0E0C0F012813F1581158179027AF0E98AF0C0E0C0F07473
:20844B00E875F087C0E0C0F090F000E0A3F5F0E0C5F012872390F000F0A3C5F0F0C5F01235
:20846B00872CC0E0C0F0740375F0001284C17FFA128666740075F000C0E0C0F0740175F041
:20848B0000C0E0C0F01280C8158115811581158179027AF0E98AF0C0E0C0F012813F1581CF
:2084AB001581740275F000C0E0C0F01284CF1581158102843F2223F42581F88682088683AA
:2084CB00080284EC78FB12865A8603088604BB0004BC00012279E5A3D9FD1BBBFFF01C80C1
:2084EB00F4128633868208868308E4FEFFE07006128633E4F022B42551A3E0B42D054307BC
:20850B0080A3E0B4300343074024D0B40A00500BCE75F00AA42EFEA3E080EEE0B46413E6E0
:20852B000886F030F708430720128733A6F018F68003B4750543070A8021B4780543071078
:20854B008019B46F104307088011128633F0A3128633A38095B462624307027A00C004C0BE
:20856B0005C006C007AB0753031F7C00E60886F01286EDA6F018F6EDD007D006D005D004EB
:20858B002430B43A0040022407C0E00AE645F070CC128633A902EF30E505742DF0A30A1251
:2085AB00863CD0E0F0A3D9FA0808EF30E7A1EAC39E509C7420F0A30A80F4B4630DAA011264
:2085CB00863312863CE6F0A380DEB47331C082C08386820886837A00E06004A30A80F986CC
:2085EB008318868212863312863C128633E0A31286336004F0A380F2D005D00480AAB469BC
:20860B001B86017A00E76004090A80F912863312863C8601E76091F009A380F8F97A0112C4
:20862B00863312863CE9809ECDC583CDCCC582CC22EE601A8FF020F715C002EAC39E500C3C
:20864B00742030F6027430F0A30A80EFD00222C82581C822C92581C97A0022D083D082CF0F
:20866B002581F581CFC082C08322CF2581F581CF2229F9E5F03AFA227C00CB30E7011CCBEE
:20868B002275F00030E70215F022FDE493A3FEE493A3FF4E7009E493FE740193FF800BE428
:2086AB0093A3B5050BE493B5F0068F838E82E473A380D81286ED8EF0ED22C0F0C0E0E5F0E7
:2086CB006C5480FF8CF030F707EB128733ACF0FBD0E0D0F030F703128733BF80051286ED29
:2086EB008046C002C001AAF0F97E007D007F11C3E933F9EA33FADF08F5F0E9D001D002229F
:20870B00ED33FDEE33FEC3ED9BF5F0EE9C40E0ADF0FED380DB12872304700205F02212878D
:20872B002C14B4FF0215F02212872CF4C5F0F4C5F0221287704029801E12877040227017D7
:20874B00801E12877040107017800C128770501080051287846009E4F5F02212878460F731
:20876B00E4F5F00422C39BC5F09C20E70720D207C345F02220D2F9D322C5F0C39C7003E5E3
:20878B00F09B2290F00CE0A360F8E0FFA3E0A3CF2582F582EF3583F58380EBFBE0CB22FC7A
:2087AB00E0FBA3E0CC22FAE0F9A3E0CA22383035315342432056312E3020202000417070F4
:2087CB006C6965642050687973696373002020202020202020202020202020200025640084
:00000001FF
